:020000004E2987
:100008000800083033190130A300A2013608840023
:1000180034089620340880044D21122884130005E2
:10002800FF3E331DA20C3319A20D3230A720A30BBB
:100038000C28220803144929A2000830331901307A
:10004800A300A20C3608840034089620340803184C
:1000580080043730A72034088004A30B2528031414
:100068004929B31C49293B28B300331C49293608C0
:100078008400340896200130A100E030A82034081C
:1000880080040130A100E030A8280830A600A700AD
:1000980037088400350833199420331D9620360814
:1000A800840034089920A001A101260803194929D0
:1000B800B3188D203608840000083405FF3EA00DD3
:1000C800A10DB31C8D20A60B5C2827083318C62861
:1000D800200849290830A600370884003508331954
:1000E8009420331D96203608840034099D20260864
:1000F800031949293318C62036088400A10CA00C1E
:1001080000083404031C340680008D20A60B8028C8
:100118004929370884003508800600008006080051
:1001280080049C28FF3A80059D288417800449296B
:10013800FF3A84178005492983178001840AFF3E06
:10014800031DA1284929A101E83EA000A109FC300E
:10015800031CB128A0070318AE28A0076400A10F4C
:10016800AE282018B728A01CBB280000BB28080010
:10017800013EA7000A30A200A3011721A70BC1283E
:1001880024080800A201A301CD28A10CA00CA20DEF
:10019800A30DFF3E0318C9282308A1002208A000C8
:1001A80049290310A00DA10DFF3E0318D5282008EA
:1001B80049290310A10CA00CFF3E0318DD282008D4
:1001C8004929A101A301A2000130F228A101A3013C
:1001D800A2000430F228A301A2000530A8002308D9
:1001E8002102031DF92822082002043003180130D7
:1001F800031902302805031DFF3049290038031D63
:10020800FF300405031DFF304929A2002008A6007D
:100218002408A0002608A4002108A6002508A1009B
:100228002608A5001929A501A4011030A600210D52
:10023800A40DA50D2208A4022308031C230FA50260
:1002480003182D292208A40723080318230FA5073C
:100258000310A00DA10DA60B1B2920084929103059
:10026800A800A101A001A70CA60C031C4129220883
:10027800A00723080318230FA107A10CA00CA50CA5
:10028800A40CA80B372924084929831303138312C4
:10029800640008008501860183168601E030850028
:1002A80083128B175A298B1B08002D2F5721831671
:1002B8008530810083125721A0308B00572181019E
:1002C800572107309F005721203084006030A1203B
:1002D800A03084005030A120203084003030A0208D
:1002E80057210A30C80057210530C7005721480850
:1002F8004707D40057216400851E8D2B57215622AD
:100308005721AA2557217025572105118316051154
:100318008312572185108316851083125721CF2405
:1003280057218515831685118312572129265721B0
:100338005308C900572129265721640050081E3C3C
:10034800031DAA298511831685118312572164007C
:1003580056085402031DB129D60157215608A0009A
:100368004808E520BE005608A0005408EA20C0004E
:100378003E08840040080221C000C1006400400813
:1003880041040319D929572101304807BE00BF018C
:10039800BF0D3E08A0003F08A1005608EF20031D2E
:1003A800D62970255721B6225721572164004908BC
:1003B80053020319F4295721D60A57215308C900B3
:1003C8005721D0015721640056084802031CF4291C
:1003D80057218515831685118312572156225721D7
:1003E80057216400851E322C57219E29572106303B
:1003F800B6000130B4000630B7000230B500013055
:10040800B3005108A000A1016E2057210800572110
:10041800992257210301CE1AFF30BE0003014E1A5C
:10042800FF30C0003E08840040080221C000C1001F
:100438006400400841040319222AD1015721080009
:100448005721992257210301CE1AFF30BE0003011C
:10045800CE19FF30C0003E08840040080221C000C9
:10046800C10064004008410403193B2AD101572107
:1004780008005721992257210301CE1AFF30BE00E8
:1004880003014E19FF30C0003E08840040080221D5
:10049800C000C1006400400841040319542AD10176
:1004A8005721080057214608A000A1010030BC20B0
:1004B800C200C301572124225721FA215721460897
:1004C800A000A1010130BC20C200C3015721242291
:1004D8005721FA215721CE1157214F08A000A10119
:1004E8000030BC20C200C30157210B225721FA213A
:1004F80057214F08A000A1010130BC20C200C30150
:1005080057210B225721FA2157214E125721061540
:1005180083160611831257210230A720572106118E
:100528008316061183125721080057214308031D1B
:10053800B42A42080B3C031CB42AA422D100B42AD2
:1005480002308A00420882073F3406345B344F3455
:1005580066346D347D3407347F346F346334393412
:1005680057210800572185118316851183125721B9
:100578000B30C200C301572199225721FA21572174
:100588000A30C200C301572199225721FA21572165
:100598003C08A0003D08A1000030BC20C200C301F7
:1005A800572199225721FA2157213C08A0003D08DC
:1005B800A1000130BC20C200C30157219922572154
:1005C800FA21572106158316061183125721023086
:1005D800A7205721061183160611831257210800F8
:1005E80057216400CE18FC2A8515831685118312BD
:1005F80057215708A000A1010030BC20C200C30148
:1006080057213D225721FA2157215708A000A1015F
:100618000130BC20C200C30157213D225721FA21D5
:1006280057214E1157214408A000A1010030BC20D9
:10063800C200C301572124225721FA215721440817
:10064800A000A1010130BC20C200C301572124220F
:100658005721FA215721CE1157214B08A000A1019B
:100668000030BC20C200C30157210B225721FA21B8
:1006780057214B08A000A1010130BC20C200C301D2
:1006880057210B225721FA2157214E1257210615BF
:1006980083160611831257210230A720572106110D
:1006A8008316061183125721080057215308A0000A
:1006B800A1010030BC20C200C301572124225721C8
:1006C800FA2157215308A000A1010130BC20C20023
:1006D800C301572124225721FA215721CE1157212E
:1006E800D1015721FA2157215408D1005721FA2165
:1006F80057214E12572106158316061183125721CA
:100708000230A7205721061183160611831257219C
:100718000800572185118316851183125721D301AB
:100728005721CE1457210630D40057214808D3004A
:100738005721592357216400851AA42B57219F2B31
:1007480057214E1657216400851EDB2B5721640064
:10075800851BBB2B57216400CE1AB32BD30A572114
:10076800640053081F3C031DBA2BD301572157219E
:100778006400051BCD2B57216400CE1AC42BD3036C
:10078800572164005308FF3C031DCC2B1E30D300B7
:10079800572157218310CE1E83148318CE16831C2D
:1007A800CE12572159235721CF245721A42B572143
:1007B8005308C80057215B30D40057214708D3009D
:1007C8005721592357216400851AEC2B5721E72B11
:1007D80057214E1657216400851E232C572164008B
:1007E800851B032C57216400CE1AFB2BD30A5721F3
:1007F800640053081F3C031D022CD30157215721C5
:100808006400051B152C57216400CE1A0C2CD30349
:10081800572164005308FF3C031D142C1E30D300DD
:10082800572157218310CE1E83148318CE16831C9C
:10083800CE12572159235721CF245721EC2B57216A
:100848005308C700572148084707D4005721CE123C
:1008580057214E125721CE10572182295721851131
:100868008316851183125721D3015721CE1457219E
:10087800562257216400851A432C57213E2C5721B4
:100888004E1657218511831685118312572164004E
:10089800851E7F2C57216400851B5F2C572164001F
:1008A800CE1A572CCF0A572164004F08183C031D55
:1008B8005E2CCF01572157216400051B712C57214D
:1008C8006400CE1A682CCF03572164004F08FF3C00
:1008D800031D702C1730CF00572157218310CE1ECF
:1008E80083148318CE16831CCE1257215622572103
:1008F800CF245721432C57214E125721CE1257216E
:10090800562257216400851A8B2C5721862C572193
:10091800CE1557218511831685118312572164003E
:10092800851EFD2C57216400851BA72C57216400C8
:10093800CE1A9F2CC60A5721640046083C3C031D6A
:10094800A62CC601572157216400051BB92C572135
:100958006400CE1AB02CC603572164004608FF3C39
:10096800031DB82C3B30C600572157218310CE1EDB
:1009780083148318CE16831CCE1257215622572172
:10098800CF2457218B2C57216400851ACD2C572151
:10099800C82C5721CE115721C201C3014208A0001B
:1009A8004308A1000D30A300AC30E720031DE42C60
:1009B80057210530A7205721C20A0319C30FD22C8B
:1009C800572108005721C201C3014208A00043086B
:1009D800A1000730A3006C30E720031DFB2C572132
:1009E8000A30A7205721C20A0319C30FE92C57213F
:1009F800080057214E125721CE1157214E11572169
:100A0800CE1257214E255721562257218515831678
:100A18008511831257216400851A142D57210F2D33
:100A280057215308CC005721132757215108D300C9
:100A380057214608CC005721132757215108C600D3
:100A480057214F08CC005721132757215108CF00B1
:100A580057214B08CC005721132757215108CB00A9
:100A680057214408CC005721132757215108C400A7
:100A780057215708CC005721132757215108D70071
:100A880057219626572129265721D6015721CE10BE
:100A980057219E2957210830850683168511831210
:100AA8005721E624572108308506831685118312BD
:100AB8005721E624572108308506831685118312AD
:100AC8005721E6245721083085068316851183129D
:100AD8005721E6245721080057210530B600103069
:100AE800B40001303820CC3020204430202035207C
:100AF80057210530B6001030B400043038200520E6
:100B0800013903194E10031D4E1435205721640076
:100B18004E1C7C2D57210530B6001030B400013032
:100B28003820CC302020BE302020352057210530F9
:100B3800B6001030B400023038200520BA00052075
:100B4800BB0035205721BE25572108005721053005
:100B5800B6001030B40001303820CC3020204E30A0
:100B68002020003020200030202031302020352067
:100B78005721080057212B30D20057216400BB1D94
:100B8800E82D57212D30D20057213A08FF3CBE00EE
:100B98003B08031C013EFF3CBF00BE0A0319BF0A05
:100BA8003E08A6003F08A7007130A2000230A3004B
:100BB8003321D5005721A3010A300921BC0021089F
:100BC800BD005721012E5721572101303A07BE0099
:100BD8003B080318013EBF007130A6000230A70091
:100BE8003E08A2003F08A3003321D5005721A301E6
:100BF8000A300921BC002108BD0057213C08A0008B
:100C08003D08A100E830A2000330A3001721240802
:100C1800BE002508BF003E08A0003F08A1006430C0
:100C2800A200A3011721B8002108B90057213C08E8
:100C3800A0003D08A100E830A2000330A30017215E
:100C4800BC002108BD00572108005721051583164F
:100C58000511831257218316051083125721053079
:100C6800B6000130B4000530B7000230B500B3015A
:100C7800BF30A000A1016E205721831605148312EE
:100C880057210530B6000130B4000530B7000230F6
:100C9800B5000130B3004920D3004920C6004920DF
:100CA800CF004920CB004920C4004920CC0049206E
:100CB800D7004920CC0057215308CC005721F426EF
:100CC80057215108D30057214608CC005721F42654
:100CD80057215108C60057214F08CC005721F42648
:100CE80057215108CF0057214B08CC005721F42633
:100CF80057215108CB0057214408CC005721F4262E
:100D080057215108C40057215708CC005721F42611
:100D180057215108D7005721051183160511831251
:100D280057210800572105158316051183125721ED
:100D380083160510831257210530B6000130B40020
:100D48000530B7000230B500B3018E30A000A10114
:100D58006E20A001A1016E205721051183160511EF
:100D6800831257210A30A72057210515831605112C
:100D7800831257210530B6000130B4000530B700A2
:100D88000230B500B301BE30A000A1016E205308A7
:100D9800A000A1016E204608A000A1016E204F0806
:100DA800A000A1016E204B08A000A1016E204408FC
:100DB800A000A1016E20A001A1016E205708A0008B
:100DC800A1016E208030A000A1016E2057210511DD
:100DD80083160511831257210A30A72057210800CE
:100DE800572170304C05CD0057214D08A000A101B6
:100DF8000430E020CD0057210F304C05C5005721A5
:100E08004D08A600A7010A30A200A3013321BE00A5
:100E18002508BF003E084507D10057210800572183
:100E28004C08A000A1010130BC20CD0057214D087D
:100E3800A0000430D820CD0057214C08A000A10103
:100E48000030BC20C50057214D084507D100572167
:100E580008006400CE18312FD00A0B110900572161
:040E68006300342FC0
:02400E00543F1D
:00000001FF
